:020000040000FA
:0600000078EF0AF0120087
:020006000000F8
:06000800C9EF07F0120031
:02000E001200DE
:020010001200DC
:0600180033EF08F01200B6
:02001E004BECA9
:1000200005F0FB0EDBCFF3FFDB06F35000090AE01F
:1000300099EC05F0FA0E04EC06F0F3E1151CF1E181
:10004000010E01D0000E7AEF05F04BEC05F03B0EEF
:10005000E12402E3E168E652E16E010EDB6A020E82
:10006000DB6AF90EDBCFF6FFFA0EDBCFF7FFFB0EF4
:10007000DBCFF8FF0800F550DF6EDF5002E19EEFA6
:1000800004F0250EDF5C02E091EF04F0030EDB6A62
:10009000040EDB6A050EDB6A060EDB6A070EDB6AFE
:1000A000B3EC04F02D0EDF5C0CE02B0EDF5C09E0FE
:1000B000200EDF5C06E0230EDF5C03E0300EDF5C29
:1000C0001AE1DF50300A14E0130A0FE0030A0AE0D5
:1000D0000B0A05E0060AE4E1030EDB80E1D7030E1C
:1000E000DB82DED7030EDB84DBD7030EDB86D8D7BB
:1000F000030EDB88D5D72A0EDF5C1BE1AFEC04F0E2
:10010000FDEC04F010E0030EDB8008680968130EB4
:10011000DBCF0DF0140EDBCF0EF0D0EC09F0040EA7
:1001200006C0DBFF03D0130EE6EC04F0B3EC04F0E2
:100130000BD0090EDB6A54EC05F003E0C8EC05F0C7
:10014000FAD7090EE6EC04F0030EDBB0DB982E0EB6
:10015000DF5C1BE1B3EC04F02A0EDF5C0BE1AFECDB
:1001600004F0FDEC04F003E1130E38EC05F0B3EC01
:1001700004F00BD0090EDB6A54EC05F003E0C8EC88
:1001800005F0FAD7090E38EC05F0680EDF5C07E1E0
:10019000B3EC04F0680EDF5C1DE1030E18D0740EA2
:1001A000DF5C17E07A0EDF5C14E0480EDF5C06E0EF
:1001B000540EDF5C03E05A0EDF5C02E1020E07D052
:1001C0006C0EDF5C03E06A0EDF5C04E1010E8BEC79
:1001D00005F0C9DBDF506E0A01E17FD31E0A01E1A1
:1001E00092D1200A01E18FD13F0A01E149D11A0AD7
:1001F00001E146D10D0A01E143D1200A01E140D1DC
:100200003A0A01E13DD1200A01E13AD1260A01E191
:1002100035D10D0A01E132D11A0A01E1D9D0200A03
:100220004AE0300A1FE0460A0EE0250A01E083D3C7
:10023000D950F90FE96EFF0EDA20EA6E010EEE5E7C
:10024000000EEE5AEE5A99EC05F0250EE66E95DB9F
:1002500003E1151C01E169D395EC05F001E26BD3D4
:10026000DB2A69D3080EDB6A040EDB50010806E2C4
:10027000040EDB045DEC05F0DB508BDB080EDB507D
:1002800009E0030EDB50010B05E172DB01E04DD309
:10029000080EDB6A64DBEFCFDFFF0DEC06F003E155
:1002A000151C01E142D395EC05F001E3DB2A60DB8C
:1002B00001E141D33AD3070EDB5002080FE1D9EC3C
:1002C00005F0030EA0EC05F00E0EEECFDBFF0F0ED7
:1002D000EECFDBFF100EEECFDBFF20D0F70EDBCF33
:1002E00017F0F80EDBCF18F0020E175E000E185A4A
:1002F000F70E17C0DBFFF80E18C0DBFF17C0E9FFD1
:1003000018C0EAFF90EC05F0166A0E0E14C0DBFF71
:100310000F0E15C0DBFF100E16C0DBFF0E0EDBCF7D
:10032000E6FF0F0EDBCFE6FF100EDBCFE6FFABECF8
:1003300009F0E552E552E552130E07C0DBFF140E3B
:1003400008C0DBFF060EDB5005E0130ED4EC05F011
:1003500001E26ADBF8EC05F002E2130E37DBBBECDE
:1003600005F006E0040ED4EC05F002E2050E2EDBEB
:10037000030EDBB005D0FCDA01E0D7D2080EDB6A51
:10038000090EDB6A0E0EDBCFF6FF0F0EDBCFF7FF99
:10039000100EDBCFF8FF0800F550DF6EDF5014E0E1
:1003A000FEEC05F011E20DEC06F003E1151C01E195
:1003B000BCD2BBDB01E3DB2A090EDB2AD9500E0FCE
:1003C000E96E000ECBDBE7D7D3DA01E1B4D2ADD2D0
:1003D000C6DA110EEECFDBFF120EEDCFDBFF110EF2
:1003E000DBCFE6FF120EDBCFE6FF9DEC09F0E55216
:1003F000E552130EF3CFDBFF140EF4CFDBFF060E36
:10040000DB5004E0130ED0DB01E20EDBF8EC05F06C
:1004100002E2130EDBDAAFDB05E0040EC5DB02E21D
:10042000050ED4DA030EDBB005D0A2DA01E07DD2EE
:10043000080EDB6A090EDB6A110EDBCFE9FF120E34
:10044000DBCFEAFFEFCFDFFFDF5014E0D7DB12E2B4
:10045000E4DB03E1151C01E168D267DB01E3DB2A81
:10046000090EDB2A110EDB2ADBCFE9FF120EE8E3CF
:10047000DB2AE6D77DDA01E15ED257D2030EDB8EAE
:10048000070EDB0410E195DB040E5ADB0A0EEECFFB
:10049000DBFF0B0EEECFDBFF0C0EEECFDBFF0D0E06
:1004A000EECFDBFF6CD0070EDB5003082CE1030E10
:1004B000DBAE0DD0B2DA020E76DAEFCF14F0156AA9
:1004C000166A176A14AE39D01568166835D0F70E5B
:1004D000DBCF15F0F80EDBCF16F0020E155E000E26
:1004E000165AF70E15C0DBFFF80E16C0DBFF15C05D
:1004F000E9FF16C0EAFFEFCF14F00A0E14C0DBFFCD
:100500000B0EDB6A38D0070EDB50020809E1030E40
:10051000DBAE04D059DB16AE10D00ED055DB0DD0BB
:10052000030EDBAE12D079DA020E3DDAF9DA166A82
:10053000176A15AE02D016681768E2DA0C0E16C0FC
:10054000DBFF0D0E17C0DBFF1AD0F70EDBCF16F066
:10055000F80EDBCF17F0020E165E000E175AF70EDC
:1005600016C0DBFFF80E17C0DBFF16C0E9FF17C08F
:10057000EAFFD6DAC5DA0C0EDB6A0D0EDB6A060E70
:10058000DB5005E1010EF36E050EF3CFDBFF150E18
:10059000DB6A160EDB6AD950370F146E000EDA20B4
:1005A000156E390E14C0DBFF3A0E15C0DBFF380E96
:1005B000DB6A080EDB6A0A0EAEDADF50780A12E058
:1005C000200A10E0280A0CE0200A0AE03F0A06E0B0
:1005D0000D0A02E0200A08E1020E05D0080E03D041
:1005E000080EDF26100E97DA030EDBBE02D0DB9278
:1005F000DB94DB50800B24E08ADAD890030EEB50BA
:10060000000A08E6000EEE5C000EEE58000EEE58F2
:10061000000EEE5815E213DA0B680C680D680E68D0
:1006200065EC09F00A0E02C0DBFF0B0E03C0DBFF16
:100630000C0E04C0DBFF0D0E05C0DBFF2D0E08D035
:10064000030EDBA202D02B0E03D0DBA408D0200EB9
:10065000F36E170EF3CFDBFF150EDB2A02D0170E59
:10066000DB6A050EDB5003E1B7D901E189D0280E22
:10067000146E150E156E000E166E070EDBCF17F0FA
:10068000186A196A1A6A17C00BF018C00CF019C062
:100690000DF01AC00EF0D3D9FDEC09F0145002246D
:1006A000F36E15500320F46E16500420F86EF4CF4C
:1006B000F7FFF3CFF6FF0800090EF5CFDBFF580E6A
:1006C000DF5C0FE1610EF36E090E7BD90AE3200EA9
:1006D000146E090EDBCFE7FF1450E75E090EE7CF7B
:1006E000DBFF070EDBCF14F0156A166A176A0FDA04
:1006F00014C00BF015C00CF016C00DF017C00EF0B2
:10070000EECF06F0EECF07F0EECF08F0EFCF09F016
:10071000FDEC09F009C0EDFF08C0EDFF07C0EDFFDB
:1007200006C0EFFF390EDBCFE9FFDB063A0EDBCF69
:10073000EAFF01E2DB06090EDBCFEFFF150EDB2A35
:100740004BD995E1030EDBA61DD06F0EDF5C06E1F1
:10075000C1D918E3150EDB285BDA14D0780EDF5C04
:1007600009E0580EDF5C06E0620EDF5C03E0420E3B
:10077000DF5C08E1020EF36E160EF3CFDBFF02D052
:10078000150EDB6A030EDB50100B0EE0040EDBCF00
:1007900014F0050EDB50D880145406E2060EDB5030
:1007A00003E1040EDB5034DA95D90AE2050EDBCF03
:1007B000E7FF150EDB50E75E050EE7CFDBFF02D04B
:1007C000050EDB6A040EDBCF14F0160E45D9D88077
:1007D000145414E2160EDBCFE6FF150EDBCFE6FF56
:1007E000040EDBCFE6FF050EDB50E552E75CE55279
:1007F000D880E754E552D880E7545FD9030EDB5028
:10080000010B0BE1080EDB5008E0B2D801E08DD0FF
:10081000080EDB50BED8080EDB6A170EDB5007E06F
:1008200088D9170EF1D903E1151C01E17ED0160E0F
:10083000DB5016E07ED9300EE66E9FD802E1151C23
:1008400074E077D9DFCFE6FF23EC09F0E552E552FB
:10085000E552F4CF15F00001F31C02E1151C65E030
:10086000050EDBCF14F0160EDB50D880145409E2CD
:10087000050EDBCFE7FF160EDB50E75E050EE7CF78
:10088000DBFF300EE66E050ECBD94FE1390EDB2AC9
:10089000DBCFE9FF3A0E01E3DB2ADBCFEAFF090EEB
:1008A000EFCFDBFFDB500EE044D9090EADD902E1FA
:1008B000151C3BE0390EDB2ADBCFE9FF3A0EEDE3F6
:1008C000DB2AEBD755D831E1160EDBCFE6FF080E59
:1008D000C3D8E552E7245DD82ED0070EDB50030ABB
:1008E0001CE0010A14E0030A07E07BD9DBCFEEFF2E
:1008F000020EDBCFEDFF1FD0F5D8196A17AE02D07C
:10090000186819682CD8BCD819C0EEFF14D0EAD8E2
:1009100017BE186824D8B4D80ED063D9DBCFEFFF48
:100920000AD07BD905E1151C03E1F368F46810D007
:10093000FCD801E3DB2A79D93AEF00F0010EDBCFD6
:1009400014F0020EDBCF15F014C0F3FF15C0F4FF56
:100950003B0EE15C02E2E16AE552E16ECBD029D9BF
:10096000020EA0EF05F061D90800F550DF6E12000D
:10097000200EE66E080E10EF06F023EC09F0E552AB
:10098000E552E552F3CF14F0F4CF15F00001F31C5B
:100990001200146E156AD950010F4DD91450EE266D
:1009A0001550ED221200185E000E195AF70E18C0ED
:1009B000DBFFF80E19C0DBFF18C0E9FF19C0EAFF22
:1009C0001200DBCFF4FFF350F45C1200DB50E76E53
:1009D000040EE7CFDBFF12000A0EDBCF14F00B0E84
:1009E000DBCF15F00C0EDBCF16F00D0EDBCF17F0C2
:1009F00014501510161017101200130EEECFDBFF57
:100A0000140EEDCFDBFF130EDBCF14F0140EDBCF93
:100A100015F00001800E15141200F70EDBCF18F050
:100A2000F80EDBCF19F01200050EDB50E66ED95040
:100A3000130F01D9E552E750EE6EED6A12000A0E6F
:100A4000DBCF06F00B0EDBCF07F00C0EDBCF08F090
:100A50000D0EDBCF09F01200DBCFE6FF150EDBCF6A
:100A6000E6FF050EDB50E552E724E552E7241200CD
:100A7000DB50CED8010EF36E060EF3CFDBFF120073
:100A8000EE50EFCFEAFFE96E16C0EEFF17C0EEFFA3
:100A900018C0EEFF1200D9CFE6FFDACFE6FFE1CFB4
:100AA000D9FFE2CFDAFF1200DFCFE6FFE66A56ECAD
:100AB0000AF0E552E552F3501200E76E080EE7CF58
:100AC000DBFF1200EECF14F0EECF15F0EFCF16F0F3
:100AD000176A1200050EDBCF14F0150EDB50D8801C
:100AE00014541200010EDBCF16F0020EDBCF17F00C
:100AF000186A1200E552E5CFDAFFE7CFD9FF1200FE
:100B00000A0E14C0DBFF0B0E15C0DBFF1200D9501C
:100B10000A0F1BEF06F0F36E070EF3CFDBFF120098
:100B2000EECF14F0EFCF15F01200010EDB2A020E0B
:100B30001200FC0EDBCFE6FFFD0EDBCFE6FF12005E
:100B4000145E000E155AF70E14C0DBFFF80E15C028
:100B5000DBFF14C0E9FF15C0EAFF1200DA20EA6EDD
:100B6000EF2AEECFF6FF000EEF22EECFF7FFEF22D7
:100B7000EECFF8FF1200040EDBCFE6FF130EDB50C2
:100B8000E552E75C9ADFDB5004DF060EDB50120013
:100B9000090EDB500A0DF350DF24D00FE76E090E6B
:100BA000E7CFDBFFB3EF04F0DB50F36E050EE1EFB0
:100BB00004F0F70EDBCF14F0F80EDBCF15F01200C7
:100BC000DFCFE6FFBDEF04F028DF030EECDE62EFBF
:100BD00005F00FEC00F0E552E552E552E552000950
:100BE0001200BDDEEE50EFCFEAFFE96E010E1200FB
:100BF000130EDB50F36E040EE1EF04F0040EDB5035
:100C0000F36E090EE1EF04F0DBCFE6FFBDEF04F079
:100C1000E76E050EE7CFDBFF12008BDFE0EF05F09C
:100C2000DBCFE6FF86DFE9EF05F0D950F90FE96E7B
:100C3000FF0EAEEF05F0E96E000EDA20EA6E12004C
:100C4000949C948E7E96190EB06EAD84AD98AC8E49
:100C5000AD9CAC9CAD9AAC889D889D8A0001A06B30
:100C6000A16BA26B1200D9CFE6FFE1CFD9FFE6520C
:100C70009E50200B01E0010E156AE85015102EE081
:100C80000001A251146E156A3F0E141810E11550A0
:100C90000EE1AD9A650EE66E140EE66E000EE66E7F
:100CA0005FD8E552E552E552AF50DF6E17D0AF5036
:100CB000E66EA151EA6A600FE96E000EEA22E55283
:100CC000E750EF6EA151146E156A3F0E141804E13F
:100CD000155002E1A16B01D0A12BA22BAC50020B4D
:100CE00001E0010E146E156A010E14180FE1155083
:100CF0000DE1AC98AC88AD9A540EE66E140EE66E1B
:100D0000000EE66E2DD8E552E552E552E552E55269
:100D1000E7CFD9FF12000001E351146E156AE451C8
:100D2000166E176A1650141802E1175015180AE0CB
:100D3000E351EA6AA30FE96E000EEA22EF50AE6EAD
:100D4000E32B1200AD50020B01E0010E146E156A88
:100D5000E8501510F7E0AD9A0001E36BE46B120068
:100D6000D9CFE6FFE1CFD9FF020EE126AD50200B2F
:100D700001E0010E156AE8501510F8E1D950FC0F9A
:100D8000146EFF0EDA20156E14C0DEFFDD6EDECFAE
:100D9000E6FFDDCFE6FFFC0EDBCFE6FFFD0EDBCF8F
:100DA000E6FFFE0EDBCFE6FFA30EE66E000EE66E5C
:100DB000DFEC08F0146E070EE15E1450A30EE66E31
:100DC000000EE66E9DEC09F0E552E552F3CFE4F03B
:100DD0000001010EE36FA351AE6EAD8A020EE15C1D
:100DE00002E2E16AE552E16EE552E7CFD9FF120077
:100DF000D9CFE6FFE1CFD9FFE652AD50200B01E09D
:100E0000010E156AE8501510F8E1FC0EDB500001E8
:100E1000E46F010EE36FDF6ADF50146E156AFC0E9B
:100E2000DB50000115AE02D0D89003D0145C000E48
:100E3000155819E2DF50E76EFD0EDBCFE9FFFE0E1D
:100E4000DBCFEAFFE750E926000EEA22EFCF14F0ED
:100E5000156ADF50EA6AA30FE96E000EEA2214C099
:100E6000EFFFDF2AD9D70001A351AE6EAD8AE5525C
:100E7000E552E7CFD9FF1200D9CFE6FFE1CFD9FF86
:100E8000E652DF6A0001A251146E156A1450151063
:100E900025E0A051EA6A600FE96E000EEA22EF50E9
:100EA000E66EDF50E76EFD0EDBCFE9FFFE0EDBCF17
:100EB000EAFFE750E926000EEA22E552E750EF6E1E
:100EC000DF2AA051146E156A3F0E141804E1155064
:100ED00002E1A06B01D0A02BA207D4D7DF50E552CE
:080EE000E552E7CFD9FF120033
:080EE8009F8A9F881200D08E42
:100EF000F28EF28C1200F250800B01E0010E176AA4
:100F0000E850171002E0000E01D0010E156AF36ED2
:100F100015C0F4FF1200F250400B01E0010E176AF9
:100F2000E850171002E0000E01D0010E156AF36EB2
:100F300015C0F4FF1200F250400B01E0010E146ED8
:100F4000156A010E141802E1155004E0D4DFF350C5
:100F5000F41002E0F36A02D0010EF36EF46A12009C
:100F6000EADFF3CF16F0F4CF17F0F350F41004E1FA
:100F7000C2DFF350F41002E0000E01D0010E156A3A
:100F8000E850151003E0010EF36E01D0F36AF46A25
:100F90001200DACFE4FFE2CFDAFFE9CFE4FFEACFD5
:100FA000E4FFF6CFE4FFF7CFE4FFF8CFE4FFF5CF9F
:100FB000E4FFF3CFE4FFF4CFE4FFFACFE4FFFBCF8D
:100FC000E4FF00EE00F0140EE80403E3EECFE4FFCC
:100FD000FBD700EE14F0070EE80403E3EECFE4FFC6
:100FE000FBD7E6529E50200B01E0010E1B6E1C6ADF
:100FF000E8501C1004E033EC06F09E9A0CD09E5092
:10100000100B01E0010E1B6E1C6AE8501C1003E07F
:101010008BEC06F09E98E55200EE1AF0070EE804FD
:1010200003E3E5CFEDFFFBD700EE13F0140EE80469
:1010300003E3E5CFEDFFFBD7E5CFFBFFE5CFFAFFFD
:10104000E5CFF4FFE5CFF3FFE5CFF5FFE5CFF8FF00
:10105000E5CFF7FFE5CFF6FFE5CFEAFFE5CFE9FF04
:10106000E5CFDAFF1100D8CFE4FFE0CFE4FFE46E74
:10107000DACFE4FFE652E552E5CFDAFFE550E5CFFF
:08108000E0FFE5CFD8FF1000EE
:08108800060EF66E000EF76E75
:10109000000EF86E00010900F550EA6F0900F550E6
:1010A000EB6F03E1EA6701D03DD00900F550E56F31
:1010B0000900F550E66F0900F550E76F09000900D7
:1010C000F550E96E0900F550EA6E090009000900C3
:1010D000F550E86F0900F550E96F09000900F6CFF7
:1010E000ECF0F7CFEDF0F8CFEEF0E5C0F6FFE6C09C
:1010F000F7FFE7C0F8FF0001E85302E1E95307E01A
:101100000900F550EE6EE807F8E2E907F9D7ECC000
:10111000F6FFEDC0F7FFEEC0F8FF0001EA07000E92
:06112000EB5BBFD71200DB
:0A112600D9CFE6FFE1CFD9FF660E36
:10113000E126DF6A010EDB6A8F0ED3147009D36ECD
:10114000FC0ED3140009D36E0F0148691F0E496FBE
:1011500020EC06F077EC07F074EC07F0420EE66E38
:10116000140EE66E000EE66EB0EC06F0E552E552A7
:10117000E552D950020FE66E000EDA20E66E3CEC26
:1011800007F0E552E552E76E010EE7CFDBFFDB50DB
:10119000146E156AE85015100EE0010EDB50E66E75
:1011A000D950020FE66E000EDA20E66EF8EC06F07B
:0E11B000E552E552E552E6683FEC0AF0D9D769
:0211BE00D9CF87
:1011C000E6FFDACFE6FFE1CFD9FFE2CFDAFFE65262
:1011D000E652F70EDBCFE6FFF80EDBCFE6FFF90EA7
:1011E000DBCFE6FFFA0EDBCFE6FFFB0EDBCFE6FF41
:1011F000D950FC0FE66EFF0EDA20E66E25EC00F00B
:10120000146E070EE15C02E2E16AE552E16E1450F1
:10121000F3CFDEFFF4CFDDFFFC0EDBCFE9FFFD0EE9
:10122000DBCFEAFFEF6ADECF14F0DDCF15F014C09C
:10123000F3FF15C0F4FFE552E552E552E5CFDAFFC2
:06124000E7CFD9FF120008
:0A124600D9CFE6FFDACFE6FFE1CFD3
:10125000D9FFE2CFDAFFFB0EDBCF14F0FC0EDBCFC1
:1012600015F00001800E15141AE1FB0EDBCFE9FF2B
:10127000FC0EDBCFEAFFEECFF3FFEDCFF4FFEE2A5B
:10128000000EEF22F3CFE9FFF4CFEAFFFD0EDBCF34
:10129000EFFFEF50156AF36E15C0F4FF10D0FB0E90
:1012A000DB50FE0806E1FD0EDBCFE6FF86EC0AF020
:1012B00005D0FD0EDBCFE6FF07EC00F0E552E5526E
:0A12C000E5CFDAFFE7CFD9FF1200F7
:0612CA0006500B02F3CFF9
:1012D00002F0F4CF03F00C02F3500326000EF420CA
:1012E000046E06500D02F3500426000EF420056E25
:1012F00006500E02F350052607500B02F35003264A
:10130000F4500422000E052207500C02F35004266C
:10131000F450052207500D02F350052608500B0229
:10132000F3500426F450052208500C02F350052611
:0A13300009500B02F35005261200CD
:06133A00FE0EE3CFE9FF07
:10134000FF0EE3CFEAFFF36AF46AEE5203E0F34ADA
:10135000F42AFBD71200FF0EE3CFF8FFE552FF0E91
:10136000E3CFF7FFE552FF0EE3CFF6FFE552E66A63
:10137000E66AE66A0900F55209E0FD0EE32A05E196
:10138000FE0EE32A02E1FF0EE32AF4D7FD0EE3CFBF
:1013900007F0FE0EE3CF08F0FF0EE3CF09F01200D6
:1013A00009C013F008C012F008500D02F4CF07F086
:1013B000F3CF06F009500E02F4CF09F0F3CF08F096
:1013C0000D02F3500726F4500822E86A0922125051
:1013D0000E02F3500726F4500822E86A09220EAEE6
:1013E000F6EF09F01250085E1350095A13AE000CC4
:0A13F0000D50085E0E50095A000C63
:0613FA00056A046A036AA3
:10140000026A200EE76ED89006360736083609368F
:1014100002360336043605360B50025C0C50035876
:101420000D5004580E50055809E30B50025E0C5045
:10143000035A0D50045A0E50055A062AE72EE4D7D7
:02144000120098
:0E1442000D0A426567696E2050726F67726115
:101450006D0D0A005541525431204F7665727275F8
:101460006E210D0A00554152543120427566666561
:0E14700072204F766572666C6F77210D0A0050
:02147E00FF0E5F
:10148000E3501E6EEF0E01D0F30EE76EE72E46EF2F
:101490000AF00C0E1D6EE76AE72E4CEF0AF01D2EC7
:0C14A0004BEF0AF01E2E44EF0AF0120081
:0414AC00F36AF46A81
:1014B000FF0EE124E96EFF0EE220EA6EED6607D032
:1014C0002F0EEF6404D03A0EEF6001D0F32A120021
:1014D000B00EF36E00EE00F00E0E01D81200EA60BE
:1014E00002D0EE6AFCD7F350E9601200EE6AFCD736
:1014F0001DEE00F02DEE00F0F86A019C44EC08F0BF
:0C15000008EC00F093EC08F0FBD71200A0
:04150C00FF0EE3509B
:10151000ADBA04D0B06AAC8EAD8A949CADA2FED7B1
:08152000AE6EF36EF46A1200D6
:0815280030313233343536371F
:09153000383961626364656600EC
:020000040001F9
:01FFF800AA5E
:01FFFA00FD09
:01FFFD00FB08
:00000001FF
